:100000008316FB28000000000B1D19289400030E26
:1000100095008312A11B1228031085190314960C56
:10002000970CA10381030B11150E8300940E140E7F
:1000300009008C00030E8D00831286160616900AA6
:100040009B1B861B26289001931F93030E08100606
:1000500003198612100D70399100110E3A200F0508
:10006000031D061206089B000B100D0E83008C0E5C
:100070000C0E0900820701340234043408341034B1
:1000800020344034803482003F3405340D34213430
:1000900010341F34223432341234213418342634CC
:1000A00030343534FF340A34083405342A343334D8
:1000B0001A34323420341E340C34FE340A340834FA
:1000C00005342A3433341E343034203435340C347F
:1000D000FE34FF348207FF34D12AFF34922AB72A34
:1000E000A92AB02AF52AFF34DD2A9E2A962AC22A96
:1000F0002C34712AFF34FF34AC299429FF34A2290F
:100100002F341F34FF34FF34FF34232A3E343F346E
:100110002E34E629FF34FF34123416343A342A34AC
:1001200018341A34FF34FF342134103438342D3469
:1001300028341D34FF34FF342334153439343D342E
:10014000202AEE29FF34FF34FF34253401340B34E8
:10015000F629022AFF34FF34262A05340D340834E8
:10016000192A102AFF34FF34322A3E2A0034762A14
:100170000A34472AFF34FF34FF347D2AFF34892AAA
:100180004E2AFF34FF343C349C290C34572AFF3468
:10019000602AFF34FF34FF346C2AFF34FF34FF340D
:1001A000FF343434FF34FF340C2BFF34D629012BB9
:1001B000FF34FF34FF34B829C029D0291D34DC298D
:1001C000CA291C347C29E92A0634302B0E34073422
:1001D000182B8C29FF34323420341E349A2AFF34F1
:1001E00035341C34FF34FF3406341A340E340734EB
:1001F0003034FF34FF34FC308500C0308600FF30DF
:1002000081000815831264007F3099008600FB305E
:100210009800850008308B009001FF308E00003080
:100220008F008B178123A401A501AB01003065214C
:100230008039A6007123E03A031956292308F03AC1
:10024000031958299030230203181A2923086A2019
:100250008400FF3A03191629A6191629040826193D
:100260003E293F398400A41B0417241B0417A41A39
:100270008417241A841704082519403A931F3E292D
:10028000261852298400AB1B5A218F128F13841B0E
:100290008F17041B8F1604083F393F3A8E00033036
:1002A00093001629FF308E008F011629A6141A29F3
:1002B00026141A292B080F39031908002B083F3977
:1002C000890004086B21AB0A080089008316081412
:1002D00083120808080088008B13831655308900A4
:1002E000AA30890088148B1788187429831266290C
:1002F000A615003426150800A513261CA517A51F52
:1003000078290830A5064223ED3047230030A5198F
:10031000FF3047236A237829A512261CA516A51E9F
:1003200078290230A5067829A6187829A413261C56
:10033000A41726188F127829A61878292413261CAA
:1003400024179929A412261CA41626188F1378297D
:100350002412261C2416A529A411261CA4157829CC
:100360002411261C241578298F10261C8F14782917
:100370003230A61C7A29B730A41F241B77307A2983
:10038000A419C7292030A61C7A29B4307A29A41EC2
:10039000C2299E2A8E30A618E229A51935307A295D
:1003A0008F30A618E229A5191E307A298630A618A2
:1003B000E229A51918307A298730A618E229A5194B
:1003C0001B307A29A41E241A7F397A29A61BE92911
:1003D0001E341E30A41F241B75307A29A61BF12958
:1003E0001B341B30A41F241B47307A29A61BFD2970
:1003F0003330A41F241B26307A293330A41F241B3A
:100400005B307A29A61B0B2A3530A41F241B7030C1
:10041000A41960307A293530A41F241B07307A29AB
:10042000A61B30343030A41F241B7230A419623054
:100430007A29A61B32343230A41F241B0F307A29AC
:10044000A61B2B341734A61B17342B34A61B2D2ABE
:100450002030A41F241B02307A292030A41F241B23
:1004600036307A29A61B392A2230A41F241B423099
:100470007A292230A41F241B37307A29A61B263460
:100480000E30A41F241B4E30A61826307A29A61B36
:100490000E344630A41F241B66307A29A61B522A2C
:1004A00073307A290F30A41F241B06307A29A61B2B
:1004B0005E2A0630A41F241B07307A2906307A29C9
:1004C000A61B672A5A30A41F241B73307A29463092
:1004D000A41F241B4F307A293630A41F241B373029
:1004E0007A294730A41F241B4F307A29A61B0234D7
:1004F0008830A41F241B80307A29A61B842A8530CB
:10050000A41F241B82307A297330A41F241B5E3061
:100510007A29A61B902A8130A41F241B8A307A29AD
:1005200060307A290615261C061178298614261CA7
:10053000861078290614261C06107829261CA22A63
:100540008615782986111810A41F1814180885001C
:100550007829A41D0334261C78294430892378295E
:10056000A41D0434261C7829533089237829A41D1E
:100570001334261C782900306521803A6B218030A5
:10058000A6067829A41D1434261C78292B080F39B7
:100590000319CF2A2B083F398900FF306B21AB01AB
:1005A0007829A41DFF34261C7829A41ADA2A0130E0
:1005B000B12378298130AB007829A41D1134261C81
:1005C0007829A41AE62A1130B12378299130AB009A
:1005D0007829A41D2734261C7829A41AF22A213050
:1005E000B1237829A130AB007829A41DB429261C99
:1005F0007829A41AFE2A3130B1237829B130AB0012
:100600007829A61C082B4330A41F241B76307A2996
:100610003330A51D43307A29A61C102B44307A298B
:100620001F30A51D44307A293030A51D1C2B7A2996
:10063000A61C142B261C78298E30A90037230A30DB
:10064000AA0029088400A223FF308E000F30AD23BA
:10065000AA0B212BCB2378291A30A51D342B7A29FC
:10066000A61C2C2B261C78298F301D2B362B83168D
:10067000051283120512080083160516831205164B
:10068000812B08008B1383168511831208008511B6
:1006900084000830A700A8010310051A4D2B85150A
:1006A000031C85110318A80A051E542B840CA70BE4
:1006B0004D2B051A592B8515281C8511051E5E2BFF
:1006C000051A602B8515051E632B051A652B051E63
:1006D000672B080083168515831285150B118B1760
:1006E00008000430AA006400A11B7C2BA90B742B0A
:1006F000AA0B742B8123712B970D960D970D160D58
:10070000A3000A30A100FF3081000B118B162308D3
:10071000080089003723090843208400FF3A0319A1
:10072000982B0408FE3A03199F2BA223890A8B2BCE
:10073000FF308E008F14AC238F103C23080048300C
:10074000AD23962B8F128F13841B8F17041B8F16CC
:1007500004083F393F3A8E0003309300931FAE2BBD
:100760000800A900FF30AA0037232908652184006A
:10077000FF3A0319CB2B04082A06031DC32BFF30B5
:100780008E000D30AD230408AA00A223A90A29086F
:100790000F39031DB52BFF308E008F013C2308005D
:1040000000000000000000000000000000000E00A2
:10420000000005002A002B000E003800300042009C
:10421000210025003F001200280008001F00FF00B9
:10422000000005002A002B000E0038001F0032009D
:10423000420025003F001200280008001E00FF0079
:10424000000005002A002B000E0038001F001F0090
:10425000420025003F001200280008001A00FF005D
:10426000000005002A002B000E0038001F001E0071
:10427000420025003F001200280008001800FF003F
:00000001FF
